 kitl

 Timestamp is 4fb04cc8 (Mon May 14 12:07:36 2012)

 Preferred load address is 10000000

 Start         Length     Name                   Class
 0001:00000000 00002138H .rdata                  CODE
 0001:00002138 00000021H .rdata$debug            CODE
 0001:0000215c 00010d50H .text                   CODE
 0001:00012eac 00000050H .xdata                  CODE
 0001:00012f00 00000031H .edata                  CODE
 0002:00000000 00005438H .data                   DATA
 0002:00005440 0004a274H .bss                    DATA
 0003:00000000 000009c8H .pdata                  DATA

  Address         Publics by Value              Rva+Base       Lib:Object

 0000:00000000       ___safe_se_handler_table   00000000     <absolute>
 0000:00000000       ___safe_se_handler_count   00000000     <absolute>
 0001:0000001c       ??_C@_1BG@JBMELNEE@?$AAU?$AAS?$AAB?$AA_?$AAS?$AAE?$AAR?$AAI?$AAA?$AAL?$AA?$AA@ 1000101c     kitl.obj
 0001:00000034       ??_C@_1BE@LBNFCPIJ@?$AAC?$AAS?$AAP?$AAS?$AAE?$AAR?$AAI?$AAA?$AAL?$AA?$AA@ 10001034     kitl.obj
 0001:00000048       ??_C@_17KDBLIHPA@?$AAF?$AAE?$AAC?$AA?$AA@ 10001048     kitl.obj
 0001:00000050       ??_C@_1BG@GIAHOCLI@?$AAU?$AAS?$AAB?$AA_?$AAR?$AAN?$AAD?$AAI?$AAS?$AA?5?$AA?$AA@ 10001050     kitl.obj
 0001:000000f8       ??_C@_05DFLKGENG@Topaz?$AA@ 100010f8     kitl.obj
 0001:00000100       ??_C@_0CA@NGKEKANM@Closing?5Handle?5of?5Timer?5Thread?6?$AA@ 10001100     kitlcore:ethdbg.obj
 0001:00000120       ??_C@_0BN@FPKBKHBK@Error?5creating?5timer?5thread?6?$AA@ 10001120     kitlcore:ethdbg.obj
 0001:00000140       ??_C@_0CF@GGNNPHKD@Connecting?5to?5Desktop?5?4?4?5resendi@ 10001140     kitlcore:ethdbg.obj
 0001:00000168       ??_C@_0BI@OFAMBHJH@Connecting?5to?5Desktop?$AN?6?$AA@ 10001168     kitlcore:ethdbg.obj
 0001:00000180       ??_C@_0EO@CEOOKDBM@?$CBKITL?5Interrupt?5thread?5got?5error@ 10001180     kitlcore:ethdbg.obj
 0001:000001d0       ??_C@_0CB@PCGPHMPD@KITL?5InterruptInitialize?5failed?6@ 100011d0     kitlcore:ethdbg.obj
 0001:000001f4       ??_C@_0BK@HDMNDFBA@KITL?5CreateEvent?5failed?$CB?6?$AA@ 100011f4     kitlcore:ethdbg.obj
 0001:00000210       ??_C@_1BK@PPDMEPMD@?$AAE?$AAd?$AAb?$AAg?$AAI?$AAn?$AAt?$AAE?$AAv?$AAe?$AAn?$AAt?$AA?$AA@ 10001210     kitlcore:ethdbg.obj
 0001:0000022c       ??_C@_0CK@GNMBECNI@?$CBDoRegisterClient?$CI?$CFs?$CJ?3?5Invalid?5p@ 1000122c     kitlcore:ethdbg.obj
 0001:00000258       ??_C@_04HIBGFPH@NULL?$AA@  10001258     kitlcore:ethdbg.obj
 0001:00000260       ??_C@_0CP@LFECMIMJ@?$CBDoRegisterClient?$CI?$CFs?$CJ?3?5Invalid?5w@ 10001260     kitlcore:ethdbg.obj
 0001:00000290       ??_C@_0DN@GDEGDLCL@?$CBKITLRegisterClient?$CI?$CFs?$CJ?3?5Client?5@ 10001290     kitlcore:ethdbg.obj
 0001:000002d0       ??_C@_0DG@FHPIAJCD@?$CBKITLRegisterClient?$CI?$CFs?$CJ?3?5No?5avai@ 100012d0     kitlcore:ethdbg.obj
 0001:00000308       ??_C@_0DO@NHOEDOMO@?$CBDoRegisterClient?$CI?$CFs?$CJ?3?5Need?5to?5s@ 10001308     kitlcore:ethdbg.obj
 0001:00000348       ??_C@_0CB@GFDDAGEF@Error?5creating?5interrupt?5thread?6@ 10001348     kitlcore:ethdbg.obj
 0001:0000036c       ??_C@_0CE@FKCJJLLC@KITL?3?5Leaving?5polling?5mode?4?4?4?50x@ 1000136c     kitlcore:ethdbg.obj
 0001:00000390       ??_C@_0DC@LLJMBDFH@?$CBKITLRegisterDfltClient?3?5Fail?5to@ 10001390     kitlcore:ethdbg.obj
 0001:000003c4       ??_C@_0DH@MFOCECCL@?$AN?6?$CBUnable?5to?5establish?5KITL?5conn@ 100013c4     kitlcore:ethdbg.obj
 0001:000003fc       ??_C@_0DN@NDJFLFHF@?$AN?6?$CBKitl?5buffer?5specified?5by?5OAL?5@ 100013fc     kitlcore:ethdbg.obj
 0001:0000043c       ??_C@_06MCCIJHBO@DBGMSG?$AA@ 1000143c     kitlcore:ethdbg.obj
 0001:00000444       ??_C@_04JMJJJNGP@PPSH?$AA@ 10001444     kitlcore:ethdbg.obj
 0001:0000044c       ??_C@_04MOKOCOLM@KDBG?$AA@ 1000144c     kitlcore:ethdbg.obj
 0001:00000454       ??_C@_0CE@HDEHCBNJ@KITL?5Error?5allocating?5timer?5memo@ 10001454     kitlcore:timer.obj
 0001:00000478       ??_C@_0DM@HHCOAHOB@?$CBKitlSendFrame?3?5transport?5failed@ 10001478     kitlcore:edbgprot.obj
 0001:000004b4       ??_C@_0CF@ELFKFCIB@?$CBSendConfig?3?5Error?5in?5KitlSendFr@ 100014b4     kitlcore:edbgprot.obj
 0001:000004dc       ??_C@_0BO@OHFCENNA@?$CBSendConfig?3?5Stack?5overflow?$AN?6?$AA@ 100014dc     kitlcore:edbgprot.obj
 0001:000004fc       ??_C@_0CM@CLKKFLBC@?$CBRetransmitFrame?3?5Error?5in?5KitlS@ 100014fc     kitlcore:edbgprot.obj
 0001:00000528       ??_C@_0CH@PDOCBOKH@?$CBKITL?3?5Error?5in?5KitlSendFrame?5fo@ 10001528     kitlcore:edbgprot.obj
 0001:00000550       ??_C@_0BP@EJOKEGGJ@?$CBSendAckNack?3?5Stack?5overflow?$AN?6?$AA@ 10001550     kitlcore:edbgprot.obj
 0001:00000570       ??_C@_0BJ@HLKLCDLN@KITL?3?5Got?5RESET?5command?6?$AA@ 10001570     kitlcore:edbgprot.obj
 0001:0000058c       ??_C@_0DH@FAHMLBID@KITL?3?5IOCTL_HAL_REBOOT?5not?5suppo@ 1000158c     kitlcore:edbgprot.obj
 0001:000005c4       ??_C@_0CM@CCHLHCID@?$CBHost?5config?5message?5size?5mismat@ 100015c4     kitlcore:edbgprot.obj
 0001:000005f0       ??_C@_0CB@MCDILJMK@?$CBKITLPollData?3?5STACK?5OVERFLOW?$CB?$AN?6@ 100015f0     kitlcore:edbgprot.obj
 0001:00000614       ??_C@_0DA@KOJGDENJ@?$CBExchangeConfig?3?5WaitForMultiple@ 10001614     kitlcore:edbgprot.obj
 0001:00000644       ??_C@_0CD@CLDOKAPO@?$CBKITLSend?3?5Error?5in?5KitlSendFram@ 10001644     kitlcore:edbgprot.obj
 0001:00000668       ??_C@_0FD@BAMAHPPH@0x?$CFx?5?$CI0x?$CFx?$CJ?3?5KITLSend?$CI?$CFu?$CJ?3?5Timed@ 10001668     kitlcore:edbgprot.obj
 0001:000006bc       ??_C@_02DKCKIIND@?$CFs?$AA@ 100016bc     kitlcore:edbgprot.obj
 0001:000006c0       ??_C@_0DD@OOGFOEID@?$CBKITLSend?$CIDBGMSG?$CJ?3?5Reentrant?5cal@ 100016c0     kitlcore:edbgprot.obj
 0001:000006f4       ??_C@_03OFAPEBGM@?$CFs?6?$AA@ 100016f4     kitlcore:edbgprot.obj
 0001:000006f8       ??_C@_0DK@DPCAMIHE@?$CBKITLSend?3?5Data?5to?5be?5send?5overl@ 100016f8     kitlcore:edbgprot.obj
 0001:00000734       ??_C@_0CJ@KPACHCHO@?$AN?6?$CBKITLRecv?3?5Invalid?5client?5ID?5?$CF@ 10001734     kitlcore:edbgprot.obj
 0001:00000760       ??_C@_0DJ@KKFBBHCF@?$CBKITLRecv?3?5Receive?5buffer?5overla@ 10001760     kitlcore:edbgprot.obj
 0001:00000b08       ??_C@_0CI@KMIJHHBB@FECInitDMABuffer?5DMA?5Buffer?5too?5@ 10001b08     oal_ethdrv_fec_common_topaz_v1:fec.obj
 0001:00000b30       ??_C@_0CB@DFINIDFK@Failed?5to?5get?5the?5external?5PHY?$AN?6@ 10001b30     oal_ethdrv_fec_common_topaz_v1:fec.obj
 0001:00000b54       ??_C@_0CN@NECAPPEM@FEC?5is?5linked?0?5speed?510?5Mbps?0?5ha@ 10001b54     oal_ethdrv_fec_common_topaz_v1:fec.obj
 0001:00000b84       ??_C@_0CN@KMHKLMCP@FEC?5is?5linked?0?5speed?510?5Mbps?0?5fu@ 10001b84     oal_ethdrv_fec_common_topaz_v1:fec.obj
 0001:00000bb4       ??_C@_0CO@NCDNBHO@FEC?5is?5linked?0?5speed?5100?5Mbps?0?5h@ 10001bb4     oal_ethdrv_fec_common_topaz_v1:fec.obj
 0001:00000be4       ??_C@_0CO@HFHJJCBN@FEC?5is?5linked?0?5speed?5100?5Mbps?0?5f@ 10001be4     oal_ethdrv_fec_common_topaz_v1:fec.obj
 0001:00000c14       ??_C@_0BG@BPBIADDC@Waiting?5for?5link?4?4?4?$AN?6?$AA@ 10001c14     oal_ethdrv_fec_common_topaz_v1:fec.obj
 0001:00000c2c       ??_C@_0BL@PCLOMCF@Initializing?5Ethernet?4?4?4?$AN?6?$AA@ 10001c2c     oal_ethdrv_fec_common_topaz_v1:fec.obj
 0001:00000cd8       ??_C@_05OHIIGEOJ@E?5?$CFx?6?$AA@ 10001cd8     oal_kitlserial_common_topaz_v1:kitlserial.obj
 0001:00000f20       ??_C@_0EH@OHHLEIM@VBridge?3?5Error?$CB?5ProduceBufferDon@ 10001f20     vbridge:vbridge.obj
 0001:00000f68       ??_C@_0ED@LALCLDGC@VBridge?3?5Error?$CB?5ConsumeBuffer?$CI?$CJ?5@ 10001f68     vbridge:vbridge.obj
 0001:00000fb0       ??_C@_0EH@PDMAJMNN@VBridge?3?5Error?$CB?5ConsumeBufferDon@ 10001fb0     vbridge:vbridge.obj
 0001:00000ff8       ??_C@_0GA@BIIJJCHI@VBridge?3?5Error?$CB?5ConsumeBufferDon@ 10001ff8     vbridge:vbridge.obj
 0001:00001058       ??_C@_08BCKMEILL@19?328?311?$AA@ 10002058     vbridge:vbridge.obj
 0001:00001064       ??_C@_0M@CJCABMIH@Sep?5?56?52006?$AA@ 10002064     vbridge:vbridge.obj
 0001:00001070       ??_C@_0CE@JNBGKBJC@VBridge?3?3?5built?5on?5?$FL?$CFs?$FN?5time?5?$FL?$CFs@ 10002070     vbridge:vbridge.obj
 0001:00001094       ??_C@_0DF@FKGFCLPJ@VBridgeInit?$CI?$CJ?4?4?4TX?5?$DN?5?$FL?$CFd?$FN?5bytes?5@ 10002094     vbridge:vbridge.obj
 0001:000010cc       ??_C@_0BO@IKIKAINA@Tx?5buffer?5?$FL0x?$CFx?$FN?5to?5?$FL0x?$CFx?$FN?4?$AN?6?$AA@ 100020cc     vbridge:vbridge.obj
 0001:000010ec       ??_C@_0BO@DMIECOA@Rx?5buffer?5?$FL0x?$CFx?$FN?5to?5?$FL0x?$CFx?$FN?4?$AN?6?$AA@ 100020ec     vbridge:vbridge.obj
 0001:0000110c       ??_C@_0CO@ILLJABOE@VBridgeKGetOneTxBuffer?$CI?$CJ?5Err?$CB?5?$FL0@ 1000210c     vbridge:vbridge.obj
 0001:0000113c       ??_C@_0DE@LOPBMMHM@VBridgeKGetOneTxBufferComplete?$CI?$CJ@ 1000213c     vbridge:vbridge.obj
 0001:00001170       ??_C@_0DJ@LKNKOIHJ@VBridgeKIndicateOneRxBuffer?$CI?$CJ?5Er@ 10002170     vbridge:vbridge.obj
 0001:000011ac       ??_C@_0DI@HEJDFJBF@?$CK?$CK?5WARNING?$CB?$CB?$CB?5?$CK?$CK?5Device?5MAC?5addr@ 100021ac     vbridge:vbridge.obj
 0001:000011e4       ??_C@_0CM@PJABNFGI@VBridge?3?3?5NK?5add?5MAC?3?5?$FL?$CFx?9?$CFx?9?$CFx?9@ 100021e4     vbridge:vbridge.obj
 0001:00001210       ??_C@_0DJ@JPHIEPAD@VBridgeKSetLocalMacAddress?$CI?$CJ?5Err@ 10002210     vbridge:vbridge.obj
 0001:0000124c       ??_C@_0DA@BNPLKEKM@VBridgeUGetOneTxPacket?$CI?$CJ?5Err?$CB?$CB?5?$FL@ 1000224c     vbridge:vbridge.obj
 0001:0000127c       ??_C@_0DI@MDDGKNHB@VBridgeUGetOneTxPacketComplete?$CI?$CJ@ 1000227c     vbridge:vbridge.obj
 0001:000012b4       ??_C@_0DA@MGPGECBI@VBridgeUGetOneRxPacket?$CI?$CJ?5Err?$CB?$CB?5?$FL@ 100022b4     vbridge:vbridge.obj
 0001:000012e4       ??_C@_0DA@KIINIKAM@VBridgeUGetOneRxPacketComplete?$CI?$CJ@ 100022e4     vbridge:vbridge.obj
 0001:00001314       ??_C@_0CD@KPODIJAL@VBridge?3?3?5RESET_BUFFER?5received?4@ 10002314     vbridge:vbridge.obj
 0001:00001338       ??_C@_0CI@BDPMFOMO@VBridge?3?3?5VB_INITIALIZED?5returns@ 10002338     vbridge:vbridge.obj
 0001:00001360       ??_C@_0DB@IMBKLANK@VBridgeUGetEDBGMac?$CI?$CJ?0?5ERR?$CB?5NULL?5@ 10002360     vbridge:vbridge.obj
 0001:00001394       ??_C@_0DB@BMKDFNPB@VBridge?3?3?5Current?5VMini?5packet?5f@ 10002394     vbridge:vbridge.obj
 0001:000013c8       ??_C@_0DG@MKNLPBLF@VBridgeUCurrentPacketFilter?$CI?$CJ?0?5E@ 100023c8     vbridge:vbridge.obj
 0001:00001490       ??_C@_0BK@FGOBGFEM@RNDISMINI?5?9?9?9?5RESET?5?9?9?9?$AN?6?$AA@ 10002490     fsl_rne_mdd_common_topaz_v1:rndis.obj
 0001:000014ac       ??_C@_0CK@HCFNMAPL@RNdis?3?3?5Too?5much?5outgoing?0?5baili@ 100024ac     fsl_rne_mdd_common_topaz_v1:rndis.obj
 0001:000014d8       ??_C@_0DK@LOJODLJL@ASSERT?$CB?5Rndis?3?3MddSendRndisMessa@ 100024d8     fsl_rne_mdd_common_topaz_v1:rndis.obj
 0001:00001514       ??_C@_0DI@ELIDGGNF@ASSERT?5Fail?5at?5uiMessageSize?$CI?$CFd?$CJ@ 10002514     fsl_rne_mdd_common_topaz_v1:rndis.obj
 0001:0000154c       ??_C@_0CK@BEACHKGH@RNdis?3?3?5No?5mem?5for?5INITIALIZE_CO@ 1000254c     fsl_rne_mdd_common_topaz_v1:rndis.obj
 0001:00001578       ??_C@_0BN@MJFOLLBM@RNdis?3?3?5Should?5not?5happen?$CB?$AN?6?$AA@ 10002578     fsl_rne_mdd_common_topaz_v1:rndis.obj
 0001:00001598       ??_C@_0CO@JHJMPDCG@RNDISMINI?5Err?$CB?$CB?5unsupported?5RNDI@ 10002598     fsl_rne_mdd_common_topaz_v1:rndis.obj
 0001:000015c8       ??_C@_0CP@HEPIJLKK@RndisMdd?3?3?5PDD?8s?5max?5RX?5buffer?5?$DN@ 100025c8     fsl_rne_mdd_common_topaz_v1:rndis.obj
 0001:000015f8       ??_C@_0CK@JCOPOCLM@ERROR?$CB?5RndisInitialize?5msg?5recei@ 100025f8     fsl_rne_mdd_common_topaz_v1:rndis.obj
 0001:00001624       ??_C@_0DB@NGCDHJGD@RndisMini?5recv?5REMOTE_NDIS_HALT_@ 10002624     fsl_rne_mdd_common_topaz_v1:rndis.obj
 0001:00001658       ??_C@_09JBPNJICM@rndis?4cpp?$AA@ 10002658     fsl_rne_mdd_common_topaz_v1:rndis.obj
 0001:00001664       ??_C@_0BP@HHOMIKAO@ASSERT?5at?5File?$CI?$CFs?$CJ?5line?5?$CI?$CFd?$CJ?$AN?6?$AA@ 10002664     fsl_rne_mdd_common_topaz_v1:rndis.obj
 0001:00001684       ??_C@_0DB@PAFHLFPB@RndisMini?5rcv?5REMOTE_NDIS_RESET_@ 10002684     fsl_rne_mdd_common_topaz_v1:rndis.obj
 0001:000016b8       ??_C@_0DA@CMCBBBCA@RNdis?3?3?5Unknown?5RNDIS?5msg?0?5buff?$FL@ 100026b8     fsl_rne_mdd_common_topaz_v1:rndis.obj
 0001:000016e8       ??_C@_0P@BDJJIKDL@Overrun?$DN0x?$CFx?6?$AN?$AA@ 100026e8     fsl_rne_mdd_common_topaz_v1:rndis.obj
 0001:000016f8       ??_C@_0BJ@IJMDONAK@Buffer?5is?5too?5big?50x?$CFx?6?$AN?$AA@ 100026f8     fsl_rne_mdd_common_topaz_v1:rndis.obj
 0001:00001714       ??_C@_0CK@LKMHPIGI@Wrong?5Data?5DataLength?5Msg?$DN0x?$CFx?0P@ 10002714     fsl_rne_mdd_common_topaz_v1:rndis.obj
 0001:00001740       ??_C@_0CN@OHNGADLJ@RNdis?3?3?5Invalid?5RndisPacket?5l?$FL?$CFd@ 10002740     fsl_rne_mdd_common_topaz_v1:rndis.obj
 0001:00001770       ??_C@_0BH@HBKBIINO@Wrong?5Data?5Type?50x?$CFx?$AN?6?$AA@ 10002770     fsl_rne_mdd_common_topaz_v1:rndis.obj
 0001:00001788       ??_C@_0CA@IBGOHNCO@Rndis?3?3?5initialization?3?5Fail?$CB?$AN?6?$AA@ 10002788     fsl_rne_mdd_common_topaz_v1:rndis.obj
 0001:000017a8       ??_C@_0CC@EELLDCCI@Rndis?3?3?5initialization?3?5Success?$AN@ 100027a8     fsl_rne_mdd_common_topaz_v1:rndis.obj
 0001:000017cc       ??_C@_0CD@EOFHIDOL@Rndis?3?3?5Get?5MAC?5address?5?$CFx?0?$CFx?0?$CFx@ 100027cc     fsl_rne_mdd_common_topaz_v1:rndis.obj
 0001:000017f0       ??_C@_0CM@KLOLOCDD@Rndis?3?3?5Err?5no?5MAC?5address?5read?5@ 100027f0     fsl_rne_mdd_common_topaz_v1:rndis.obj
 0001:0000181c       ??_C@_0BL@EINAHMEI@Rndis?3?3?5PDDInit?5Success?$CB?$AN?6?$AA@ 1000281c     fsl_rne_mdd_common_topaz_v1:rndis.obj
 0001:00001838       ??_C@_0BK@BFGGBGMH@Rndis?3?3?5initialization?$CB?$AN?6?$AA@ 10002838     fsl_rne_mdd_common_topaz_v1:rndis.obj
 0001:00001854       ??_C@_0CI@PFDJABBD@Rndis?3?3?5Address?5static?5map?5to?5ad@ 10002854     fsl_rne_mdd_common_topaz_v1:rndis.obj
 0001:0000187c       ??_C@_0CH@LBCKJEJO@Rndis?3?3?5initialization?3?5with?5add@ 1000287c     fsl_rne_mdd_common_topaz_v1:rndis.obj
 0001:00001938       ??_C@_0BP@JDIDIKNB@OID?$FL?$CFx?$FN?5not?5yet?5implemented?$CB?$AN?6?$AA@ 10002938     fsl_rne_mdd_common_topaz_v1:hostmini.obj
 0001:00001958       ??_C@_0CP@MKNOHPIM@HostMini?3?3?5New?5filter?5set?3?5?$FL0x?$CFx@ 10002958     fsl_rne_mdd_common_topaz_v1:hostmini.obj
 0001:00001988       ??_C@_0BE@LPGPNKBH@HostMiniInit?3?3?5?$CB?$CB?$AN?6?$AA@ 10002988     fsl_rne_mdd_common_topaz_v1:hostmini.obj
 0001:00001a30       ??_C@_1O@NJEHEHHO@?$AAu?$AAt?$AAi?$AAl?$AA?4?$AAc?$AA?$AA@ 10002a30     fsl_rne_mdd_common_topaz_v1:util.obj
 0001:00001a40       ??_C@_1FA@PHGBNLGM@?$AAM?$AAi?$AAc?$AAr?$AAo?$AAs?$AAo?$AAf?$AAt?$AA?5?$AAR?$AAN?$AAD?$AAI?$AAS?$AA?5?$AAK?$AAI?$AAT?$AAL?$AA?5?$AAf?$AAo?$AAr?$AA?5?$AAF?$AAS?$AAL?$AA?5?$AAH?$AAS?$AA?5@ 10002a40     fsl_rne_pdd_common_topaz_v1:rndis_pdd.obj
 0001:00001a90       ??_C@_1BE@DEAPIJA@?$AAM?$AAi?$AAc?$AAr?$AAo?$AAs?$AAo?$AAf?$AAt?$AA?$AA@ 10002a90     fsl_rne_pdd_common_topaz_v1:rndis_pdd.obj
 0001:00001b4c       DigitTable                 10002b4c     fsl_rne_pdd_common_topaz_v1:rndis_pdd.obj
 0001:00001b70       ??_C@_0BO@FJNCJEJP@Discard?5?$CFd?5Pending?5Messages?$AN?6?$AA@ 10002b70     fsl_rne_pdd_common_topaz_v1:rndis_pdd.obj
 0001:00001b90       ??_C@_1BC@GDFGLIEL@?$AAO?$AAT?$AAG?$AAG?$AAr?$AAo?$AAu?$AAp?$AA?$AA@ 10002b90     usb_usbfn_mx25_topaz_v1:i_pdd.obj
 0001:00001ba4       ??_C@_1BG@HHFAGDDC@?$AAO?$AAT?$AAG?$AAS?$AAu?$AAp?$AAp?$AAo?$AAr?$AAt?$AA?$AA@ 10002ba4     usb_usbfn_mx25_topaz_v1:i_pdd.obj
 0001:00001bbc       ??_C@_1BI@BHLBGEOK@?$AAP?$AAr?$AAi?$AAo?$AAr?$AAi?$AAt?$AAy?$AA2?$AA5?$AA6?$AA?$AA@ 10002bbc     usb_usbfn_mx25_topaz_v1:i_pdd.obj
 0001:00001bd4       ??_C@_17DJGGJCGD@?$AAI?$AAr?$AAq?$AA?$AA@ 10002bd4     usb_usbfn_mx25_topaz_v1:i_pdd.obj
 0001:00001bdc       ??_C@_1O@LBBNFMDB@?$AAM?$AAe?$AAm?$AAL?$AAe?$AAn?$AA?$AA@ 10002bdc     usb_usbfn_mx25_topaz_v1:i_pdd.obj
 0001:00001bec       ??_C@_1BA@INLDIDEN@?$AAM?$AAe?$AAm?$AAB?$AAa?$AAs?$AAe?$AA?$AA@ 10002bec     usb_usbfn_mx25_topaz_v1:i_pdd.obj
 0001:00001d20       ??_C@_1BM@LGGJJGMB@?$AAP?$AAr?$AAi?$AAm?$AAe?$AAF?$AAZ?$AAL?$AAT?$AA?3?$AA?5?$AA?$CF?$AAs?$AA?$AA@ 10002d20     usb_usbfn_mx25_topaz_v1:i_pdd.obj
 0001:00001d3c       ??_C@_17HCEMPBGG@?$AAO?$AAU?$AAT?$AA?$AA@ 10002d3c     usb_usbfn_mx25_topaz_v1:i_pdd.obj
 0001:00001d44       ??_C@_15BNKBCKPG@?$AAI?$AAN?$AA?$AA@ 10002d44     usb_usbfn_mx25_topaz_v1:i_pdd.obj
 0001:00001d50       ??_C@_1EA@GOCNCOIC@?$AAI?$AAs?$AAs?$AAu?$AAe?$AAT?$AAr?$AAa?$AAn?$AAs?$AAf?$AAe?$AAr?$AA?3?$AA?5?$AA?$CF?$AAs?$AA?5?$AAw?$AAi?$AAt?$AAh?$AA?5?$AA?$CF?$AAd?$AA?5?$AAb?$AAy?$AAt?$AAe?$AAs?$AA?$AA@ 10002d50     usb_usbfn_mx25_topaz_v1:i_pdd.obj
 0001:00001d90       ??_C@_1DA@JMEFNML@?$AAA?$AAb?$AAo?$AAr?$AAt?$AAT?$AAr?$AAa?$AAn?$AAs?$AAf?$AAe?$AAr?$AA?5?$AA?$CI?$AA?$CF?$AAs?$AA?5?$AAE?$AAP?$AA?$CF?$AAd?$AA?$CJ?$AA?$AA@ 10002d90     usb_usbfn_mx25_topaz_v1:i_pdd.obj
 0001:00001dc0       ??_C@_19CIJIHAKK@?$AAN?$AAU?$AAL?$AAL?$AA?$AA@ 10002dc0     usb_usbfn_mx25_topaz_v1:i_pdd.obj
 0001:00001dcc       ??_C@_1CA@HMLLGPGC@?$AA?9?$AAS?$AAe?$AAn?$AAd?$AAC?$AAS?$AAH?$AA?5?$AA?$CI?$AAE?$AAP?$AA?$CF?$AAd?$AA?$CJ?$AA?$AA@ 10002dcc     usb_usbfn_mx25_topaz_v1:i_pdd.obj
 0001:00001dec       ??_C@_1CA@DFPEHIFN@?$AA?$CL?$AAS?$AAe?$AAn?$AAd?$AAC?$AAS?$AAH?$AA?5?$AA?$CI?$AAE?$AAP?$AA?$CF?$AAd?$AA?$CJ?$AA?$AA@ 10002dec     usb_usbfn_mx25_topaz_v1:i_pdd.obj
 0001:00001e0c       ??_C@_1CI@HKDMKLGF@?$AAD?$AAe?$AAt?$AAa?$AAc?$AAh?$AA?3?$AA?5?$AAP?$AAO?$AAR?$AAT?$AAS?$AAC?$AA?5?$AA0?$AAx?$AA?$CF?$AAx?$AA?$AA@ 10002e0c     usb_usbfn_mx25_topaz_v1:i_pdd.obj
 0001:00001e34       ??_C@_1O@BJIMCIMK@?$AAR?$AAe?$AAs?$AAu?$AAm?$AAe?$AA?$AA@ 10002e34     usb_usbfn_mx25_topaz_v1:i_pdd.obj
 0001:00001e44       ??_C@_1BE@JNFMNJIM@?$AAI?$AAn?$AAt?$AAr?$AA?3?$AAD?$AAo?$AAn?$AAe?$AA?$AA@ 10002e44     usb_usbfn_mx25_topaz_v1:i_pdd.obj
 0001:00001e58       ??_C@_1EE@JAFGGGNF@?$AAI?$AAn?$AAt?$AAr?$AA?3?$AAU?$AAI?$AA?5?$AAS?$AAE?$AAT?$AAU?$AAP?$AAS?$AAT?$AAA?$AAT?$AA?5?$AA?$CF?$AAx?$AA?5?$AAE?$AAN?$AAD?$AAP?$AAT?$AAC?$AAO?$AAM?$AAP?$AA?5?$AA?$CF@ 10002e58     usb_usbfn_mx25_topaz_v1:i_pdd.obj
 0001:00001e9c       ??_C@_1BC@MCOFDLFC@?$AAI?$AAn?$AAt?$AAr?$AA?3?$AAS?$AAL?$AAI?$AA?$AA@ 10002e9c     usb_usbfn_mx25_topaz_v1:i_pdd.obj
 0001:00001eb0       ??_C@_1BO@EGKDOEEI@?$AAI?$AAn?$AAt?$AAr?$AA?3?$AAS?$AAi?$AAg?$AAn?$AAa?$AAl?$AAl?$AAe?$AAd?$AA?$AA@ 10002eb0     usb_usbfn_mx25_topaz_v1:i_pdd.obj
 0001:00001ff0       ??_C@_0CB@KKLHFGEJ@OALStall?3?5EPIT?5mapping?5failed?$CB?$AN?6@ 10002ff0     ethdrv:ethdrv.obj
 0001:00002164       OEMKitlStartup             10003164 f   kitl.obj
 0001:00002318       OALSerialInit              10003318 f   kitl.obj
 0001:00002378       OEMKitlSerialInit          10003378 f   kitl.obj
 0001:000023d4       OALGetTickCount            100033d4 f   kitl.obj
 0001:00002408       OALClockSetGatingMode      10003408 f   kitl.obj
 0001:00002464       IsDesktopDbgrExist         10003464 f   kitlcore:ethdbg.obj
 0001:00002520       ChkDfltSvc                 10003520 f   kitlcore:ethdbg.obj
 0001:00002770       KITLDeregisterClient       10003770 f   kitlcore:ethdbg.obj
 0001:00002a28       KITLWriteDebugString       10003a28 f   kitlcore:ethdbg.obj
 0001:00002f60       KITLInitializeInterrupt    10003f60 f   kitlcore:ethdbg.obj
 0001:000030d8       KITLRegisterDfltClient     100040d8 f   kitlcore:ethdbg.obj
 0001:000033ec       KitlInit                   100043ec f   kitlcore:ethdbg.obj
 0001:00003448       KITLRegisterClient         10004448 f   kitlcore:ethdbg.obj
 0001:0000366c       ExtKITLIoctl               1000466c f   kitlcore:ethdbg.obj
 0001:00003a08       KITLIoctl                  10004a08 f   kitlcore:ethdbg.obj
 0001:00003c84       KitlDllMain                10004c84 f   kitlcore:ethdbg.obj
 0001:00003fb0       KITLOutputDebugString      10004fb0 f   kitlcore:debug.obj
 0001:0000404c       InitTimerList              1000504c f   kitlcore:timer.obj
 0001:00004088       FreeTimerEntry             10005088 f   kitlcore:timer.obj
 0001:000040e0       TimerCallback              100050e0 f   kitlcore:timer.obj
 0001:000042b0       TimerStart                 100052b0 f   kitlcore:timer.obj
 0001:00004394       TimerStop                  10005394 f   kitlcore:timer.obj
 0001:0000448c       CancelTimersForClient      1000548c f   kitlcore:timer.obj
 0001:000044dc       KitlSetTimerCallback       100054dc f   kitlcore:timer.obj
 0001:00004588       TimerThread                10005588 f   kitlcore:timer.obj
 0001:00004720       DoDebugBreak               10005720 f   kitlcore:edbgprot.obj
 0001:00004728       ResetClientState           10005728 f   kitlcore:edbgprot.obj
 0001:000047e4       KitlSendRawData            100057e4 f   kitlcore:edbgprot.obj
 0001:000048ac       KitlSendFrame              100058ac f   kitlcore:edbgprot.obj
 0001:0000491c       SendConfig                 1000591c f   kitlcore:edbgprot.obj
 0001:00004a5c       RetransmitFrame            10005a5c f   kitlcore:edbgprot.obj
 0001:000054c0       HandleRecvInterrupt        100064c0 f   kitlcore:edbgprot.obj
 0001:00005640       KITLPollResponse           10006640 f   kitlcore:edbgprot.obj
 0001:000057a0       ExchangeConfig             100067a0 f   kitlcore:edbgprot.obj
 0001:000058a4       KITLSend                   100068a4 f   kitlcore:edbgprot.obj
 0001:00005ec0       KITLRecv                   10006ec0 f   kitlcore:edbgprot.obj
 0001:00006274       NKSetLastError             10007274 f   nkstub:nkstub.obj
 0001:00006298       NKGetLastError             10007298 f   nkstub:nkstub.obj
 0001:000062bc       EnterCriticalSection       100072bc f   nkstub:nkstub.obj
 0001:000062e0       LeaveCriticalSection       100072e0 f   nkstub:nkstub.obj
 0001:00006304       InitializeCriticalSection  10007304 f   nkstub:nkstub.obj
 0001:00006328       DeleteCriticalSection      10007328 f   nkstub:nkstub.obj
 0001:0000634c       INTERRUPTS_OFF             1000734c f   nkstub:nkstub.obj
 0001:00006370       INTERRUPTS_ENABLE          10007370 f   nkstub:nkstub.obj
 0001:00006394       NKSetInterruptEvent        10007394 f   nkstub:nkstub.obj
 0001:000063b8       NKSleep                    100073b8 f   nkstub:nkstub.obj
 0001:000063dc       NKCreateStaticMapping      100073dc f   nkstub:nkstub.obj
 0001:00006400       NKForceCleanBoot           10007400 f   nkstub:nkstub.obj
 0001:00006424       NKUnicodeToAscii           10007424 f   nkstub:nkstub.obj
 0001:00006448       NKPhysToVirt               10007448 f   nkstub:nkstub.obj
 0001:0000646c       NKVirtToPhys               1000746c f   nkstub:nkstub.obj
 0001:00006490       __report_gsfailure         10007490 f   nkstub:nkstub.obj
 0001:000064b4       OEMWriteDebugByte          100074b4 f   oemstub:oemstub.obj
 0001:000064d8       OEMGetTickCount            100074d8 f   oemstub:oemstub.obj
 0001:000064fc       OEMInterruptEnable         100074fc f   oemstub:oemstub.obj
 0001:00006520       OEMIoControl               10007520 f   oemstub:oemstub.obj
 0001:00006578       OALKitlInit                10007578 f   oal_kitl:kitl.obj
 0001:00006600       OALKitlPowerOff            10007600 f   oal_kitl:kitl.obj
 0001:0000666c       OALKitlPowerOn             1000766c f   oal_kitl:kitl.obj
 0001:000066cc       OEMKitlInit                100076cc f   oal_kitl:kitl.obj
 0001:0000674c       OALKitlCreateName          1000774c f   oal_kitl:name.obj
 0001:0000683c       OEMKitlIoctl               1000783c f   oal_kitl:kitlioctl.obj
 0001:00006864       OALKitlFindDevice          10007864 f   oal_kitl:device.obj
 0001:00006dd0       OALKitlSerialInit          10007dd0 f   oal_kitl:kitlserial.obj
 0001:00007a6c       DecodeIP                   10008a6c f   oal_kitl:kitleth.obj
 0001:00007fa4       OALIoCtlVBridge            10008fa4 f   oal_kitl:kitleth.obj
 0001:0000837c       OALKitlEthInit             1000937c f   oal_kitl:kitleth.obj
 0001:00008654       MIIREAD                    10009654 f   oal_ethdrv_fec_common_topaz_v1:fec.obj
 0001:000086d4       MIIWRITE                   100096d4 f   oal_ethdrv_fec_common_topaz_v1:fec.obj
 0001:00008738       CalculateHashValue         10009738 f   oal_ethdrv_fec_common_topaz_v1:fec.obj
 0001:00008788       FECEnableInts              10009788 f   oal_ethdrv_fec_common_topaz_v1:fec.obj
 0001:000087a0       FECDisableInts             100097a0 f   oal_ethdrv_fec_common_topaz_v1:fec.obj
 0001:000087b8       FECInitDMABuffer           100097b8 f   oal_ethdrv_fec_common_topaz_v1:fec.obj
 0001:00008940       FECInit                    10009940 f   oal_ethdrv_fec_common_topaz_v1:fec.obj
 0001:00008d44       FECSendFrame               10009d44 f   oal_ethdrv_fec_common_topaz_v1:fec.obj
 0001:00008e20       FECGetFrame                10009e20 f   oal_ethdrv_fec_common_topaz_v1:fec.obj
 0001:00008f58       FECCurrentPacketFilter     10009f58 f   oal_ethdrv_fec_common_topaz_v1:fec.obj
 0001:00008fb4       FECMulticastList           10009fb4 f   oal_ethdrv_fec_common_topaz_v1:fec.obj
 0001:0000905c       SerialInit                 1000a05c f   oal_kitlserial_common_topaz_v1:kitlserial.obj
 0001:00009098       SerialDeinit               1000a098 f   oal_kitlserial_common_topaz_v1:kitlserial.obj
 0001:0000909c       SerialRecv                 1000a09c f   oal_kitlserial_common_topaz_v1:kitlserial.obj
 0001:0000910c       SerialSend                 1000a10c f   oal_kitlserial_common_topaz_v1:kitlserial.obj
 0001:00009160       SerialSendComplete         1000a160 f   oal_kitlserial_common_topaz_v1:kitlserial.obj
 0001:00009164       SerialEnableInts           1000a164 f   oal_kitlserial_common_topaz_v1:kitlserial.obj
 0001:00009168       SerialDisableInts          1000a168 f   oal_kitlserial_common_topaz_v1:kitlserial.obj
 0001:0000916c       OALPAtoVA                  1000a16c f   oal_memory_arm:memory.obj
 0001:0000919c       OALVAtoPA                  1000a19c f   oal_memory_arm:memory.obj
 0001:000091d8       OALArgsQuery               1000a1d8 f   args:args.obj
 0001:0000930c       OALConfigSerialUART        1000a30c f   serialutils:serialutils.obj
 0001:000094d4       OALConfigSerialIOMUX       1000a4d4 f   serialutils:serialutils.obj
 0001:00009540       OALKitlFECBSPInit          1000a540 f   bspfec:bspfec.obj
 0001:000096bc       BSPFECusesRMII             1000a6bc f   bspfec:bspfec.obj
 0001:000096c4       ProduceBuffer              1000a6c4 f   vbridge:vbridge.obj
 0001:000097dc       ProduceBufferDone          1000a7dc f   vbridge:vbridge.obj
 0001:0000981c       ConsumeBuffer              1000a81c f   vbridge:vbridge.obj
 0001:000098e0       ConsumeBufferDone          1000a8e0 f   vbridge:vbridge.obj
 0001:00009970       VBridgeInit                1000a970 f   vbridge:vbridge.obj
 0001:00009a84       VBridgeKGetOneTxBuffer     1000aa84 f   vbridge:vbridge.obj
 0001:00009af8       VBridgeKGetOneTxBufferComplete 1000aaf8 f   vbridge:vbridge.obj
 0001:00009b44       VBridgeKIndicateOneRxBuffer 1000ab44 f   vbridge:vbridge.obj
 0001:00009c34       VBridgeKSetLocalMacAddress 1000ac34 f   vbridge:vbridge.obj
 0001:00009cb4       VBridgeUGetOneTxPacket     1000acb4 f   vbridge:vbridge.obj
 0001:00009d10       VBridgeUGetOneTxPacketComplete 1000ad10 f   vbridge:vbridge.obj
 0001:00009d54       VBridgeUGetOneRxPacket     1000ad54 f   vbridge:vbridge.obj
 0001:00009da8       VBridgeUGetOneRxPacketComplete 1000ada8 f   vbridge:vbridge.obj
 0001:00009de4       VBridgeUWildCard           1000ade4 f   vbridge:vbridge.obj
 0001:00009e78       VBridgeUGetEDBGMac         1000ae78 f   vbridge:vbridge.obj
 0001:00009ec0       VBridgeUCurrentPacketFilter 1000aec0 f   vbridge:vbridge.obj
 0001:00009f08       __GSHandlerCheckCommon     1000af08 f   fulllibc:gshandler.obj
 0001:00009f44       __GSHandlerCheck           1000af44 f   fulllibc:gshandler.obj
 0001:00009f68       memset                     1000af68 f   fulllibc:memset.obj
 0001:00009ff0       __security_check_cookie    1000aff0 f   fulllibc:armsecgs.obj
 0001:0000a004       __gsfailure                1000b004 f   fulllibc:armsecgs.obj
 0001:0000a048       __rt_udiv                  1000b048 f   fulllibc:__udiv.obj
 0001:0000a10c       strcpy                     1000b10c f   fulllibc:strcpy.obj
 0001:0000a190       strlen                     1000b190 f   fulllibc:mdsstrlen.obj
 0001:0000a1f4       strcmp                     1000b1f4 f   fulllibc:mdsstrcmp.obj
 0001:0000a2e4       memcpy                     1000b2e4 f   fulllibc:memcpy.obj
 0001:0000a690       memcpybigblk               1000b690 f   fulllibc:memcpy.obj
 0001:0000b044       __C_specific_handler       1000c044 f   fulllibc:chandler.obj
 0001:0000b190       __GSHandlerCheck_SEH       1000c190 f   fulllibc:gshandlerseh.obj
 0001:0000b1e0       __rt_sdiv                  1000c1e0 f   fulllibc:__div.obj
 0001:0000b2bc       memcmp                     1000c2bc f   fulllibc:memcmp.obj
 0001:0000b388       __raise_int_divide_by_zero 1000c388 f   fulllibc:diverr.obj
 0001:0000b3ac       __C_ExecuteTerminationHandler 1000c3ac f   fulllibc:jmpuwind.obj
 0001:0000b3ac       __C_ExecuteExceptionFilter 1000c3ac f   fulllibc:jmpuwind.obj
 0001:0000b3ec       __crtRaiseException        1000c3ec f   fulllibc:raiseexc.obj
 0001:0000b408       RndisRestart               1000c408 f   fsl_rne_mdd_common_topaz_v1:rndis.obj
 0001:0000b470       RndisPrepareRndisPacket    1000c470 f   fsl_rne_mdd_common_topaz_v1:rndis.obj
 0001:0000b518       MddSendRndisPacketComplete 1000c518 f   fsl_rne_mdd_common_topaz_v1:rndis.obj
 0001:0000b52c       RndisEDbgSendFrame         1000c52c f   fsl_rne_mdd_common_topaz_v1:rndis.obj
 0001:0000b674       MddSendRndisMessageComplete 1000c674 f   fsl_rne_mdd_common_topaz_v1:rndis.obj
 0001:0000b6a0       RndisSendRndisMessage      1000c6a0 f   fsl_rne_mdd_common_topaz_v1:rndis.obj
 0001:0000b8c4       RndisProcessMessage        1000c8c4 f   fsl_rne_mdd_common_topaz_v1:rndis.obj
 0001:0000bc64       RndisEDbgGetFrame          1000cc64 f   fsl_rne_mdd_common_topaz_v1:rndis.obj
 0001:0000bdb4       RndisProcessPacket         1000cdb4 f   fsl_rne_mdd_common_topaz_v1:rndis.obj
 0001:0000bf04       RndisInit                  1000cf04 f   fsl_rne_mdd_common_topaz_v1:rndis.obj
 0001:0000c120       RndisCurrentPacketFilter   1000d120 f   fsl_rne_mdd_common_topaz_v1:rndis.obj
 0001:0000c124       RndisMulticastList         1000d124 f   fsl_rne_mdd_common_topaz_v1:rndis.obj
 0001:0000c12c       RndisEnableInts            1000d12c f   fsl_rne_mdd_common_topaz_v1:rndis.obj
 0001:0000c158       RndisDisableInts           1000d158 f   fsl_rne_mdd_common_topaz_v1:rndis.obj
 0001:0000c184       HostMiniQueryInformation   1000d184 f   fsl_rne_mdd_common_topaz_v1:hostmini.obj
 0001:0000c474       HostMiniSetInformation     1000d474 f   fsl_rne_mdd_common_topaz_v1:hostmini.obj
 0001:0000c5c0       MddIndicateRndisMessage    1000d5c0 f   fsl_rne_mdd_common_topaz_v1:hostmini.obj
 0001:0000c5d0       MddIndicateRndisPacket     1000d5d0 f   fsl_rne_mdd_common_topaz_v1:hostmini.obj
 0001:0000c5f0       MDDAllocDataWrapper        1000d5f0 f   fsl_rne_mdd_common_topaz_v1:hostmini.obj
 0001:0000c618       MDDFreeMem                 1000d618 f   fsl_rne_mdd_common_topaz_v1:hostmini.obj
 0001:0000c61c       MDDFreeDataWrapper         1000d61c f   fsl_rne_mdd_common_topaz_v1:hostmini.obj
 0001:0000c630       HostMiniInit               1000d630 f   fsl_rne_mdd_common_topaz_v1:hostmini.obj
 0001:0000c674       InitBuffer                 1000d674 f   fsl_rne_mdd_common_topaz_v1:util.obj
 0001:0000c710       AvaiableBufferSize         1000d710 f   fsl_rne_mdd_common_topaz_v1:util.obj
 0001:0000c74c       AllocBuffer                1000d74c f   fsl_rne_mdd_common_topaz_v1:util.obj
 0001:0000c83c       FreeBuffer                 1000d83c f   fsl_rne_mdd_common_topaz_v1:util.obj
 0001:0000c9b8       GetFirstUsedBuffer         1000d9b8 f   fsl_rne_mdd_common_topaz_v1:util.obj
 0001:0000cab0       PDD_GetDescriptor          1000dab0 f   fsl_rne_pdd_common_topaz_v1:rndis_pdd.obj
 0001:0000cc1c       PDD_DoVendorCommand        1000dc1c f   fsl_rne_pdd_common_topaz_v1:rndis_pdd.obj
 0001:0000cd38       setupDataOutTransfer       1000dd38 f   fsl_rne_pdd_common_topaz_v1:rndis_pdd.obj
 0001:0000ce04       HandleSetupPacket          1000de04 f   fsl_rne_pdd_common_topaz_v1:rndis_pdd.obj
 0001:0000d128       PDD_SendRndisMessage       1000e128 f   fsl_rne_pdd_common_topaz_v1:rndis_pdd.obj
 0001:0000d1bc       PDD_SendRndisPacket        1000e1bc f   fsl_rne_pdd_common_topaz_v1:rndis_pdd.obj
 0001:0000d26c       PDD_Set                    1000e26c f   fsl_rne_pdd_common_topaz_v1:rndis_pdd.obj
 0001:0000d344       PDD_Get                    1000e344 f   fsl_rne_pdd_common_topaz_v1:rndis_pdd.obj
 0001:0000d418       PDD_ISR                    1000e418 f   fsl_rne_pdd_common_topaz_v1:rndis_pdd.obj
 0001:0000d438       PDD_IndicateRndisPacketComplete 1000e438 f   fsl_rne_pdd_common_topaz_v1:rndis_pdd.obj
 0001:0000d460       SetRNDISSerialNumber       1000e460 f   fsl_rne_pdd_common_topaz_v1:rndis_pdd.obj
 0001:0000d504       NotifyHandler              1000e504 f   fsl_rne_pdd_common_topaz_v1:rndis_pdd.obj
 0001:0000d914       PDDInit                    1000e914 f   fsl_rne_pdd_common_topaz_v1:rndis_pdd.obj
 0001:0000e2fc       UfnPdd_PowerDown           1000f2fc f   usb_usbfn_mx25_topaz_v1:i_pdd.obj
 0001:0000e3a4       UfnPdd_PowerUp             1000f3a4 f   usb_usbfn_mx25_topaz_v1:i_pdd.obj
 0001:0000e45c       UpdateDevicePower          1000f45c f   usb_usbfn_mx25_topaz_v1:i_pdd.obj
 0001:0000e518       SetupEvent                 1000f518 f   usb_usbfn_mx25_topaz_v1:i_pdd.obj
 0001:0000e660       CopyFromUncachedBuffer     1000f660 f   usb_usbfn_mx25_topaz_v1:i_pdd.obj
 0001:0000ea24       UfnPdd_IssueTransfer       1000fa24 f   usb_usbfn_mx25_topaz_v1:i_pdd.obj
 0001:0000efe4       UfnPdd_AbortTransfer       1000ffe4 f   usb_usbfn_mx25_topaz_v1:i_pdd.obj
 0001:0000f17c       UfnPdd_StallEndpoint       1001017c f   usb_usbfn_mx25_topaz_v1:i_pdd.obj
 0001:0000f1f8       UfnPdd_ClearEndpointStall  100101f8 f   usb_usbfn_mx25_topaz_v1:i_pdd.obj
 0001:0000f288       UfnPdd_IsEndpointHalted    10010288 f   usb_usbfn_mx25_topaz_v1:i_pdd.obj
 0001:0000f2f4       UfnPdd_SendControlStatusHandshake 100102f4 f   usb_usbfn_mx25_topaz_v1:i_pdd.obj
 0001:0000f378       UfnPdd_InitiateRemoteWakeup 10010378 f   usb_usbfn_mx25_topaz_v1:i_pdd.obj
 0001:0000f380       SetPowerState              10010380 f   usb_usbfn_mx25_topaz_v1:i_pdd.obj
 0001:0000f3cc       UfnPdd_IOControl           100103cc f   usb_usbfn_mx25_topaz_v1:i_pdd.obj
 0001:0000f5e0       UfnPdd_Deinit              100105e0 f   usb_usbfn_mx25_topaz_v1:i_pdd.obj
 0001:0000f5f4       UfnPdd_DeregisterDevice    100105f4 f   usb_usbfn_mx25_topaz_v1:i_pdd.obj
 0001:0000f5fc       UfnPdd_Stop                100105fc f   usb_usbfn_mx25_topaz_v1:i_pdd.obj
 0001:0000f66c       UfnPdd_DeinitEndpoint      1001066c f   usb_usbfn_mx25_topaz_v1:i_pdd.obj
 0001:0000f700       UfnPdd_InitEndpoint        10010700 f   usb_usbfn_mx25_topaz_v1:i_pdd.obj
 0001:0000f814       UfnPdd_SetAddress          10010814 f   usb_usbfn_mx25_topaz_v1:i_pdd.obj
 0001:0000f84c       UfnPdd_Start               1001084c f   usb_usbfn_mx25_topaz_v1:i_pdd.obj
 0001:0000f940       UfnPdd_RegisterDevice      10010940 f   usb_usbfn_mx25_topaz_v1:i_pdd.obj
 0001:0000fb70       UfnPdd_IsEndpointSupportable 10010b70 f   usb_usbfn_mx25_topaz_v1:i_pdd.obj
 0001:0000fb8c       UfnPdd_IsConfigurationSupportable 10010b8c f   usb_usbfn_mx25_topaz_v1:i_pdd.obj
 0001:0000fce4       UfnPdd_Init                10010ce4 f   usb_usbfn_mx25_topaz_v1:i_pdd.obj
 0001:0000ffe0       CheckEndpoint              10010fe0 f   usb_usbfn_mx25_topaz_v1:i_pdd.obj
 0001:000104a0       InterruptHandle            100114a0 f   usb_usbfn_mx25_topaz_v1:i_pdd.obj
 0001:00010a50       FslUfnGetUsbFnPdd          10011a50 f   usb_usbfn_eboot_mx25_topaz_v1:i_stub.obj
 0001:00010a5c       FslUfnRequestIrq           10011a5c f   usb_usbfn_eboot_mx25_topaz_v1:i_stub.obj
 0001:00010a64       FslUfnIsUSBKitlEnable      10011a64 f   usb_usbfn_eboot_mx25_topaz_v1:i_stub.obj
 0001:00010a6c       FslUfnCreateThread         10011a6c f   usb_usbfn_eboot_mx25_topaz_v1:i_stub.obj
 0001:00010a74       UsbFnInterruptThread       10011a74 f   usb_usbfn_eboot_mx25_topaz_v1:i_stub.obj
 0001:00010a9c       FslUfnTrigIrq              10011a9c f   usb_usbfn_eboot_mx25_topaz_v1:i_stub.obj
 0001:00010ac4       FslUfnDeinit               10011ac4 f   usb_usbfn_eboot_mx25_topaz_v1:i_stub.obj
 0001:00010ac8       FslUfnGetDMABuffer         10011ac8 f   usb_usbfn_eboot_mx25_topaz_v1:i_stub.obj
 0001:00010b48       BSPUSBClockSwitch          10011b48 f   usb_usbfn_eboot_mx25_topaz_v1:i_stub.obj
 0001:00010b50       BSPUSBClockCreateFileMapping 10011b50 f   usb_usbfn_eboot_mx25_topaz_v1:i_stub.obj
 0001:00010b58       GetDeviceRegistryParams    10011b58 f   usb_usbfn_eboot_mx25_topaz_v1:i_stub.obj
 0001:00010b78       SetInterruptEvent          10011b78 f   usb_usbfn_eboot_mx25_topaz_v1:i_stub.obj
 0001:00010bac       FslUfnGetPageNumber        10011bac f   usb_usbfn_eboot_mx25_topaz_v1:i_stub.obj
 0001:00010bcc       FslUfnGetPageSize          10011bcc f   usb_usbfn_eboot_mx25_topaz_v1:i_stub.obj
 0001:00010bd4       FslUfnGetPageShift         10011bd4 f   usb_usbfn_eboot_mx25_topaz_v1:i_stub.obj
 0001:00010bdc       FslInitializeCriticalSection 10011bdc f   usb_usbfn_eboot_mx25_topaz_v1:i_stub.obj
 0001:00010be0       FslEnterCriticalSection    10011be0 f   usb_usbfn_eboot_mx25_topaz_v1:i_stub.obj
 0001:00010be4       FslLeaveCriticalSection    10011be4 f   usb_usbfn_eboot_mx25_topaz_v1:i_stub.obj
 0001:00010be8       CreateBusAccessHandle      10011be8 f   usb_usbfn_eboot_mx25_topaz_v1:i_stub.obj
 0001:00010bf0       CeLogData                  10011bf0 f   usb_usbfn_eboot_mx25_topaz_v1:i_stub.obj
 0001:00010bf4       MmMapIoSpace               10011bf4 f   usb_usbfn_eboot_mx25_topaz_v1:i_stub.obj
 0001:00010c08       InterruptDisable           10011c08 f   usb_usbfn_eboot_mx25_topaz_v1:i_stub.obj
 0001:00010c0c       CacheSync                  10011c0c f   usb_usbfn_eboot_mx25_topaz_v1:i_stub.obj
 0001:00010c20       LockPages                  10011c20 f   usb_usbfn_eboot_mx25_topaz_v1:i_stub.obj
 0001:00010c3c       GetLastError               10011c3c f   usb_usbfn_eboot_mx25_topaz_v1:i_stub.obj
 0001:00010c44       UnlockPages                10011c44 f   usb_usbfn_eboot_mx25_topaz_v1:i_stub.obj
 0001:00010c4c       CeOpenCallerBuffer         10011c4c f   usb_usbfn_eboot_mx25_topaz_v1:i_stub.obj
 0001:00010c58       CeCloseCallerBuffer        10011c58 f   usb_usbfn_eboot_mx25_topaz_v1:i_stub.obj
 0001:00010c60       StringCchLengthW           10011c60 f   usb_usbfn_eboot_mx25_topaz_v1:i_stub.obj
 0001:00010c74       StringCchVPrintfW          10011c74 f   usb_usbfn_eboot_mx25_topaz_v1:i_stub.obj
 0001:00010c7c       SetDevicePowerState        10011c7c f   usb_usbfn_eboot_mx25_topaz_v1:i_stub.obj
 0001:00010c84       Sleep                      10011c84 f   usb_usbfn_eboot_mx25_topaz_v1:i_stub.obj
 0001:00010c88       CacheRangeFlush            10011c88 f   usb_usbfn_eboot_mx25_topaz_v1:i_stub.obj
 0001:00010fc8       ?HandleGetDescriptor@@YAXPAU_USB_DEVICE_REQUEST@@PAU_EP0_REQUEST@@@Z 10011fc8 f   fsl_serial_pdd_common_topaz_v1:serial_dl.obj
 0001:00011058       ?HandleTransferComplete@@YAXPAU_STransfer@@@Z 10012058 f   fsl_serial_pdd_common_topaz_v1:serial_dl.obj
 0001:00011420       USBSerialInit              10012420 f   fsl_serial_pdd_common_topaz_v1:serial_dl.obj
 0001:000114fc       OEMSerialSendRaw           100124fc f   fsl_serial_pdd_common_topaz_v1:serial_dl.obj
 0001:000115e4       USBKitlSerialInit          100125e4 f   fsl_serial_pdd_common_topaz_v1:serial_dl.obj
 0001:000115fc       USBKitlSerialRecv          100125fc f   fsl_serial_pdd_common_topaz_v1:serial_dl.obj
 0001:000116d0       USBKitlSerialSend          100126d0 f   fsl_serial_pdd_common_topaz_v1:serial_dl.obj
 0001:000116f4       USBKitlSerialEnableInts    100126f4 f   fsl_serial_pdd_common_topaz_v1:serial_dl.obj
 0001:000116f8       USBKitlSerialDisableInts   100126f8 f   fsl_serial_pdd_common_topaz_v1:serial_dl.obj
 0001:000116fc       OALFlushDCache             100126fc f   oal_cache_arm926:flushdc.obj
 0001:00011708       OALCleanDCache             10012708 f   oal_cache_arm926:cleandc.obj
 0001:00011714       OALFlushDCacheLines        10012714 f   oal_cache_arm926:flushdclines.obj
 0001:00011734       OALStall                   10012734 f   ethdrv:ethdrv.obj
 0001:00011858       OEMKitlGetSecs             10012858 f   ethdrv:ethdrv.obj
 0001:00011938       memmove                    10012938 f   fulllibc:memmove.obj
 0001:000120c8       memmovebigblk              100130c8 f   fulllibc:memmove.obj
 0001:00012b60       __rt_udivrem64by64         10013b60 f   fulllibc:mdsdiv64.obj
 0001:00012c58       __rt_divrem64by64          10013c58 f   fulllibc:mdsdiv64.obj
 0001:00012ca8       __rt_udiv64by64            10013ca8 f   fulllibc:mdsdiv64.obj
 0001:00012cb8       __rt_urem64by64            10013cb8 f   fulllibc:mdsdiv64.obj
 0001:00012cd0       __rt_sdiv64by64            10013cd0 f   fulllibc:mdsdiv64.obj
 0001:00012ce0       __rt_srem64by64            10013ce0 f   fulllibc:mdsdiv64.obj
 0001:00012cf8       GetRNDISMACAddress         10013cf8 f   fsl_usbfn_rndiskitl_mx25_topaz_v1:hwinit.obj
 0001:00012d2c       controllerSetup            10013d2c f   fsl_usbfn_rndiskitl_mx25_topaz_v1:hwinit.obj
 0001:00012db0       HardwareInitialize         10013db0 f   fsl_usbfn_rndiskitl_mx25_topaz_v1:hwinit.obj
 0001:00012e58       PowerDownSchemeExist       10013e58 f   fsl_usbfn_rndiskitl_mx25_topaz_v1:hwinit.obj
 0001:00012e60       BSPUsbXvrEnableVBUSIntr    10013e60 f   fsl_usbfn_rndiskitl_mx25_topaz_v1:hwinit.obj
 0001:00012e7c       BSPUsbResetPHY             10013e7c f   fsl_usbfn_rndiskitl_mx25_topaz_v1:hwinit.obj
 0001:00012e80       BSPUsbSetBusConfig         10013e80 f   fsl_usbfn_rndiskitl_mx25_topaz_v1:hwinit.obj
 0001:00012e90       BSPUSBInterruptControl     10013e90 f   fsl_usbfn_rndiskitl_mx25_topaz_v1:hwinit.obj
 0001:00012e94       BSPPhyShowDevDiscon        10013e94 f   fsl_usbfn_rndiskitl_mx25_topaz_v1:hwinit.obj
 0001:00012e9c       BSPUsbSetCurrentLimitation 10013e9c f   fsl_usbfn_rndiskitl_mx25_topaz_v1:hwinit.obj
 0001:00012ea0       FslUfnGetKitlDMABuffer     10013ea0 f   fsl_usbfn_rndiskitl_mx25_topaz_v1:stub.obj
 0002:00000120       g_dwKITLThreadPriority     10014120     kitlcore:ethdbg.obj
 0002:00000124       g_dwKITLTimerThreadPriority 10014124     kitlcore:ethdbg.obj
 0002:00000128       __security_cookie          10014128     nkstub:nkstub.obj
 0002:0000012c       __security_cookie_complement 1001412c     nkstub:nkstub.obj
 0002:00000130       Am79c874Info               10014130     oal_ethdrv_fec_common_topaz_v1:fec.obj
 0002:00000334       PhyInfo                    10014334     oal_ethdrv_fec_common_topaz_v1:fec.obj
 0002:00000348       LAN8700Info                10014348     oal_ethdrv_fec_common_topaz_v1:fec.obj
 0002:00000550       Dp83640Info                10014550     oal_ethdrv_fec_common_topaz_v1:fec.obj
 0002:00000758       KSZ8041NLInfo              10014758     oal_ethdrv_fec_common_topaz_v1:fec.obj
 0002:0000095c       bRndisSendPacketEmpty      1001495c     fsl_rne_mdd_common_topaz_v1:rndis.obj
 0002:00000990       RNdisMddSupportedOids      10014990     fsl_rne_mdd_common_topaz_v1:hostmini.obj
 0002:00000a20       g_InterruptData            10014a20     fsl_rne_pdd_common_topaz_v1:rndis_pdd.obj
 0002:00001000       g_rndis_ep2_buf            10015000     fsl_rne_pdd_common_topaz_v1:buffer.obj
 0002:00001000       g_serial_rev_buf           10015000     fsl_rne_pdd_common_topaz_v1:buffer.obj
 0002:00003000       g_serial_send_buf          10017000     fsl_rne_pdd_common_topaz_v1:buffer.obj
 0002:00003000       g_rndis_ep3_buf            10017000     fsl_rne_pdd_common_topaz_v1:buffer.obj
 0002:00005000       g_rndis_ep0_buf            10019000     fsl_rne_pdd_common_topaz_v1:buffer.obj
 0002:0002adbc       dwCurrentPacketFilter      1003edbc     vbridge:vbridge.obj
 0002:0002adc0       bValidAddress              1003edc0     vbridge:vbridge.obj
 0002:0002adc4       bWarnNoMacDone             1003edc4     vbridge:vbridge.obj
 0002:0002adc8       g_bResetBuffer             1003edc8     vbridge:vbridge.obj
 0002:0002adcc       g_bUOpened                 1003edcc     vbridge:vbridge.obj
 0002:00034ca8       g_pEP3DataWrapper          10048ca8     fsl_rne_pdd_common_topaz_v1:rndis_pdd.obj
 0002:00034cac       g_devState                 10048cac     fsl_rne_pdd_common_topaz_v1:rndis_pdd.obj
 0002:00034cb0       g_EP0TransferState         10048cb0     fsl_rne_pdd_common_topaz_v1:rndis_pdd.obj
 0002:00034cb4       g_EP2TransferState         10048cb4     fsl_rne_pdd_common_topaz_v1:rndis_pdd.obj
 0002:00036040       ?g_mddInterface@@3U_UFN_MDD_INTERFACE_INFO@@A 1004a040     fsl_serial_pdd_common_topaz_v1:serial_dl.obj
 0002:00036048       ?g_EP1Transfer@@3U_STransfer@@A 1004a048     fsl_serial_pdd_common_topaz_v1:serial_dl.obj
 0002:00036068       ?g_RecvBuffer@@3PAEA       1004a068     fsl_serial_pdd_common_topaz_v1:serial_dl.obj
 0002:00036088       ?g_pddInterface@@3U_UFN_PDD_INTERFACE_INFO@@A 1004a088     fsl_serial_pdd_common_topaz_v1:serial_dl.obj
 0002:000360e8       ?g_EP2Transfer@@3U_STransfer@@A 1004a0e8     fsl_serial_pdd_common_topaz_v1:serial_dl.obj
 0002:00036108       ?g_EP0Transfer@@3U_STransfer@@A 1004a108     fsl_serial_pdd_common_topaz_v1:serial_dl.obj
 0002:0003616c       ?g_DeviceState@@3W4DEVICE_STATE@@A 1004a16c     fsl_serial_pdd_common_topaz_v1:serial_dl.obj
 0002:00036170       ?g_EP0State@@3W4TRANSFER_STATE@@A 1004a170     fsl_serial_pdd_common_topaz_v1:serial_dl.obj
 0002:00036174       ?g_EP1State@@3W4TRANSFER_STATE@@A 1004a174     fsl_serial_pdd_common_topaz_v1:serial_dl.obj
 0002:00036178       ?g_EP2State@@3W4TRANSFER_STATE@@A 1004a178     fsl_serial_pdd_common_topaz_v1:serial_dl.obj
 0002:0003617c       ?g_RecvBufferHead@@3GA     1004a17c     fsl_serial_pdd_common_topaz_v1:serial_dl.obj
 0002:00036180       ?g_RecvBufferTail@@3GA     1004a180     fsl_serial_pdd_common_topaz_v1:serial_dl.obj
 0002:000361a4       g_KitlInterval             1004a1a4     <common>
 0002:000361c0       preallocent                1004a1c0     <common>
 0002:00036454       g_pprcNK                   1004a454     <common>
 0002:00036460       DfltClnts                  1004a460     <common>
 0002:00036600       g_kpriv                    1004a600     <common>
 0002:00036660       TimerListCS                1004a660     <common>
 0002:00036674       KITLGlobalState            1004a674     <common>
 0002:00036680       SendFmtBuf                 1004a680     <common>
 0002:00036c80       KITLcs                     1004ac80     <common>
 0002:00036c94       g_pKData                   1004ac94     <common>
 0002:00036ca0       KITLODScs                  1004aca0     <common>
 0002:00036cc0       KITLKCallcs                1004acc0     <common>
 0002:00036ce0       Kitl                       1004ace0     <common>
 0002:00036d40       KITLClients                1004ad40     <common>
 0002:00036f40       g_oalCacheInfo             1004af40     <common>
 0002:00036f88       g_pNKGlobal                1004af88     <common>
 0002:00036f8c       g_pOemGlobal               1004af8c     <common>
 0002:00036fa0       g_oalKitlBuffer            1004afa0     <common>
 0002:00046fa0       g_UUID                     1005afa0     <common>
 0002:00046fb0       g_pBSPArgs                 1005afb0     <common>
 0002:00046fb4       pucRxMax                   1005afb4     <common>
 0002:00046fb8       pucTxConsumer              1005afb8     <common>
 0002:00046fbc       pucTxMin                   1005afbc     <common>
 0002:00046fc0       TxBuffers                  1005afc0     <common>
 0002:0004afc4       pucRxProducer              1005efc4     <common>
 0002:0004afc8       EDBGMacAddress             1005efc8     <common>
 0002:0004afd0       pucTxMax                   1005efd0     <common>
 0002:0004afd4       pucRxMin                   1005efd4     <common>
 0002:0004afd8       pucTxProducer              1005efd8     <common>
 0002:0004afdc       pucRxConsumer              1005efdc     <common>
 0002:0004afe0       RxBuffers                  1005efe0     <common>
 0002:0004f000       RndisMdd                   10063000     <common>
 0002:0004f0d0       g_EP0DataWrapper           100630d0     <common>
 0002:0004f0e0       MDDZONE5                   100630e0     <common>
 0002:0004f0e8       g_mddInterface             100630e8     <common>
 0002:0004f100       g_EP1Transfer              10063100     <common>
 0002:0004f120       g_RndisKitlDev             10063120     <common>
 0002:0004f568       g_udr                      10063568     <common>
 0002:0004f570       MDDZONE4                   10063570     <common>
 0002:0004f574       PDDZONE                    10063574     <common>
 0002:0004f580       g_EP3Transfer              10063580     <common>
 0002:0004f5a0       g_pddInterface             100635a0     <common>
 0002:0004f600       MDDZONE3                   10063600     <common>
 0002:0004f620       g_EP2Transfer              10063620     <common>
 0002:0004f640       PDDZONE0                   10063640     <common>
 0002:0004f660       g_EP0Transfer              10063660     <common>
 0002:0004f680       MDDZONE0                   10063680     <common>
 0002:0004f684       MDDZONE                    10063684     <common>
 0002:0004f688       MDDZONE2                   10063688     <common>
 0002:0004f6a0       g_csRegister               100636a0     <common>

 entry point at        0001:00003c84

 Static symbols

 0001:00002478       NewClient                  10003478 f   kitlcore:ethdbg.obj
 0001:00002568       RegisterClientPart2        10003568 f   kitlcore:ethdbg.obj
 0001:000028b4       ChkCnxDsktp                100038b4 f   kitlcore:ethdbg.obj
 0001:000028c8       TranCnxDsktp               100038c8 f   kitlcore:ethdbg.obj
 0001:000028f8       KITLConnectToDesktop       100038f8 f   kitlcore:ethdbg.obj
 0001:00002abc       MemCopyUserPtr             10003abc f   kitlcore:ethdbg.obj
 0001:00002b58       KITLInterruptThread        10003b58 f   kitlcore:ethdbg.obj
 0001:00002d14       DoRegisterClient           10003d14 f   kitlcore:ethdbg.obj
 0001:00003234       StartKitl                  10004234 f   kitlcore:ethdbg.obj
 0001:00003d34       pOutputByte                10004d34 f   kitlcore:debug.obj
 0001:00003d64       pOutputNumHex              10004d64 f   kitlcore:debug.obj
 0001:00003dac       pOutputNumDecimal          10004dac f   kitlcore:debug.obj
 0001:00003df0       vOutputFormatString        10004df0 f   kitlcore:debug.obj
 0001:000041fc       TimerListInsert            100051fc f   kitlcore:timer.obj
 0001:000047b8       CheckCfg                   100057b8 f   kitlcore:edbgprot.obj
 0001:000047cc       ChkAck                     100057cc f   kitlcore:edbgprot.obj
 0001:00004b50       SendAckNack                10005b50 f   kitlcore:edbgprot.obj
 0001:00004c50       ProcessAdminMsg            10005c50 f   kitlcore:edbgprot.obj
 0001:00004fb4       RetransmitCfg              10005fb4 f   kitlcore:edbgprot.obj
 0001:00004fc8       TranAck                    10005fc8 f   kitlcore:edbgprot.obj
 0001:00005034       ProcessRecvFrame           10006034 f   kitlcore:edbgprot.obj
 0001:000055ac       KITLPollData               100065ac f   kitlcore:edbgprot.obj
 0001:00006998       SerialSend                 10007998 f   oal_kitl:kitlserial.obj
 0001:00006a2c       SerialRecv                 10007a2c f   oal_kitl:kitlserial.obj
 0001:00006cb0       SerialEncode               10007cb0 f   oal_kitl:kitlserial.obj
 0001:00006d60       SerialDecode               10007d60 f   oal_kitl:kitlserial.obj
 0001:00006d78       SerialEnableInt            10007d78 f   oal_kitl:kitlserial.obj
 0001:00006db8       SerialGetDevCfg            10007db8 f   oal_kitl:kitlserial.obj
 0001:00006dc8       SerialSetHostCfg           10007dc8 f   oal_kitl:kitlserial.obj
 0001:00006fa8       Sum                        10007fa8 f   oal_kitl:kitleth.obj
 0001:00007010       SendARP                    10008010 f   oal_kitl:kitleth.obj
 0001:000070d8       EncodeIP                   100080d8 f   oal_kitl:kitleth.obj
 0001:0000723c       EncodeUDP                  1000823c f   oal_kitl:kitleth.obj
 0001:00007328       SendDHCP                   10008328 f   oal_kitl:kitleth.obj
 0001:00007518       RenewDHCP                  10008518 f   oal_kitl:kitleth.obj
 0001:00007554       DecodeDHCP                 10008554 f   oal_kitl:kitleth.obj
 0001:00007798       DecodeICMP                 10008798 f   oal_kitl:kitleth.obj
 0001:000078c8       DecodeUDP                  100088c8 f   oal_kitl:kitleth.obj
 0001:00007b40       KitlEthDecode              10008b40 f   oal_kitl:kitleth.obj
 0001:00007c5c       KitlEthEncode              10008c5c f   oal_kitl:kitleth.obj
 0001:00007ca4       KitlEthSetHostCfg          10008ca4 f   oal_kitl:kitleth.obj
 0001:00007cac       KitlEthGetDevCfg           10008cac f   oal_kitl:kitleth.obj
 0001:00007d58       KitlEthSend                10008d58 f   oal_kitl:kitleth.obj
 0001:00007e6c       KitlEthRecv                10008e6c f   oal_kitl:kitleth.obj
 0001:00007f64       KitlEthEnableInt           10008f64 f   oal_kitl:kitleth.obj
 0001:00008134       GetAddressDHCP             10009134 f   oal_kitl:kitleth.obj
 0001:0000ca44       PDD_SendNotification       1000da44 f   fsl_rne_pdd_common_topaz_v1:rndis_pdd.obj
 0001:0000ca70       PDD_RecvNotification       1000da70 f   fsl_rne_pdd_common_topaz_v1:rndis_pdd.obj
 0001:0000cf80       RegisterUSBDevice          1000df80 f   fsl_rne_pdd_common_topaz_v1:rndis_pdd.obj
 0001:0000db24       CeLogMsg                   1000eb24 f   usb_usbfn_mx25_topaz_v1:i_pdd.obj
 0001:0000dbcc       GetSetupPacket             1000ebcc f   usb_usbfn_mx25_topaz_v1:i_pdd.obj
 0001:0000dc70       InitQh0                    1000ec70 f   usb_usbfn_mx25_topaz_v1:i_pdd.obj
 0001:0000df54       PrimeQh0ForZeroTransfer    1000ef54 f   usb_usbfn_mx25_topaz_v1:i_pdd.obj
 0001:0000e190       HandleUSBReset             1000f190 f   usb_usbfn_mx25_topaz_v1:i_pdd.obj
 0001:0000e75c       BuildTdBufferList          1000f75c f   usb_usbfn_mx25_topaz_v1:i_pdd.obj
 0001:00010cf8       ?HandleUSBDeviceRegistration@@YAXXZ 10011cf8 f   fsl_serial_pdd_common_topaz_v1:serial_dl.obj
 0001:00011168       ?HandleSetupPkt@@YAXPAU_USB_DEVICE_REQUEST@@PAU_EP0_REQUEST@@@Z 10012168 f   fsl_serial_pdd_common_topaz_v1:serial_dl.obj
 0001:00011298       ?HandlePDDNotification@@YAHPAXKK@Z 10012298 f   fsl_serial_pdd_common_topaz_v1:serial_dl.obj
